:020000040800F2
:1000000000060020E1020008E3020008E302000805
:10001000E3020008E3020008E3020008E30200082C
:10002000E3020008E3020008E3020008BD34000810
:10003000E3020008E3020008E3020008E30200080C
:10004000E3020008E3020008E3020008E3020008FC
:10005000E3020008E3020008A5380008D1380008D0
:10006000FD3800082939000855390008E302000866
:10007000E3020008E3020008E3020008E3020008CC
:10008000E3020008E3020008E3020008E3020008BC
:10009000E3020008E3020008E302000881390008D7
:1000A000E3020008E3020008E3020008E30200089C
:1000B000E3020008E3020008E3020008E30200088C
:1000C000E3020008E3020008E3020008E30200087C
:1000D000E3020008E3020008E3020008E30200086C
:1000E000E5390008E3020008E3020008E302000823
:1000F000E3020008E3020008E3020008E30200084C
:10010000E3020008E3020008593A0008E30200088D
:10011000E3020008E3020008E3020008E30200082B
:10012000E3020008E3020008E3020008E30200081B
:10013000E3020008E3020008E3020008E30200080B
:10014000E3020008E3020008E3020008E3020008FB
:10015000E3020008E3020008E3020008E3020008EB
:10016000E3020008E3020008E3020008E3020008DB
:10017000E30200083D2E0008E3020008E302000845
:10018000E3020008E3020008E3020008E3020008BB
:10019000E3020008E3020008E3020008E3020008AB
:1001A000E3020008E3020008E3020008E30200089B
:1001B000E3020008E3020008E3020008E30200088B
:1001C000E3020008E3020008E3020008E30200087B
:1001D000E3020008292E0008E3020008E3020008F9
:1001E000E3020008E3020008E3020008E30200085B
:1001F000E3020008E3020008E3020008E30200084B
:10020000E3020008E3020008E3020008E30200083A
:10021000E3020008E3020008E3020008E30200082A
:10022000E3020008E3020008E3020008E30200081A
:10023000E3020008E3020008E3020008E30200080A
:10024000E3020008E3020008E3020008E3020008FA
:10025000E3020008E3020008E3020008E3020008EA
:10026000E3020008E3020008E3020008E3020008DA
:10027000E3020008E3020008E3020008E3020008CA
:10028000E3020008E3020008E3020008E3020008BA
:10029000E3020008E3020008E3020008E3020008AA
:1002A000E3020008E3020008E3020008E30200089A
:1002B000E3020008E3020008E3020008E30200088A
:1002C000E3020008E3020008E3020008E30200087A
:1002D000E3020008E3020008E3020008E30200086A
:1002E00002E000F000F8FEE772B6374880F30888B5
:1002F000364880F3098836483649086040F20000E5
:10030000CCF200004EF63471CEF200010860BFF36B
:100310004F8FBFF36F8F40F20000C0F2F0004EF637
:100320008851CEF200010860BFF34F8FBFF36F8F8B
:100330004FF00000E1EE100A4EF63C71CEF20001E3
:100340000860062080F31488BFF36F8F01F0E2FF8E
:1003500003F006F84FF055301F491B4A91423CBF4D
:1003600041F8040BFAE71D49184A91423CBF41F895
:10037000040BFAE71A491B4A1B4B9A423EBF51F83D
:10038000040B42F8040BF8E700201849184A914280
:100390003CBF41F8040BFAE701F0FAFF03F064F800
:1003A000144C154DAC4203DA54F8041B8847F9E7A6
:1003B00000F042F8114C124DAC4203DA54F8041B21
:1003C0008847F9E701F0E2BF000600200022002084
:1003D0000000000808ED00E00000002000060020FA
:1003E000383E0008002200205C220020602200200D
:1003F00034430020E0020008E0020008E0020008A8
:10040000E00200082DE9F04F2DED108AC1F80CD064
:10041000D0F80CD0BDEC108ABDE8F08F002383F338
:1004200011882846A047002001F0FAFAFEE701F003
:1004300089FA00DFFEE7000038B500F0DBFB01F0D1
:1004400029FF054601F05CFF0446D0B90F4B9D42E1
:1004500019D001339D4241F2883512BF0446002570
:100460000124002001F020FF0CB100F077F800F02B
:1004700073FD00F025FC284600F01EF900F06EF830
:10048000F9E70025EDE70546EBE700BF010007B0FF
:1004900008B500F0E7FBA0F120035842584108BD21
:1004A00007B541F21203022101A8ADF8043000F0B3
:1004B000F7FB03B05DF804FB38B5302383F31188F4
:1004C000174803680BB101F077FB0023154A4FF47E
:1004D0007A71134801F066FB002383F31188124CF4
:1004E000236813B12368013B2360636813B1636819
:1004F000013B63600D4D2B7833B963687BB90220F3
:1005000000F0A4FC322363602B78032B07D16368CF
:100510002BB9022000F09AFC4FF47A73636038BD67
:1005200060220020B90400088023002078220020E7
:10053000084B187003280CD8DFE800F00805020803
:10054000022000F07BBC022000F06EBC024B0022B7
:100550005A6070477822002080230020F8B5504B65
:10056000504A1C461968013100F0998004339342C7
:10057000F8D162684C4B9A4240F291804B4B9B6899
:1005800003F1006303F500339A4280F08880002075
:1005900000F0BCFB0220FFF7CBFF454B0021D3F856
:1005A000E820C3F8E810D3F81021C3F81011D3F8ED
:1005B0001021D3F8EC20C3F8EC10D3F81421C3F8C1
:1005C0001411D3F81421D3F8F020C3F8F010D3F8A5
:1005D0001821C3F81811D3F81821D3F8802042F05D
:1005E0000062C3F88020D3F8802022F00062C3F8B4
:1005F0008020D3F88020D3F8802042F00072C3F826
:100600008020D3F8802022F00072C3F88020D3F835
:10061000803072B64FF0E023C3F8084DD4E90004EF
:10062000BFF34F8FBFF36F8F224AC2F88410BFF31E
:100630004F8F536923F480335361BFF34F8FD2F848
:10064000803043F6E076C3F3C905C3F34E335B0154
:1006500003EA060C29464CEA81770139C2F8747224
:10066000F9D2203B13F1200FF2D1BFF34F8FBFF32C
:100670006F8FBFF34F8FBFF36F8F536923F4003336
:1006800053610023C2F85032BFF34F8FBFF36F8F17
:10069000302383F31188854680F308882047F8BD0E
:1006A0000000020820000208FFFF010800220020CD
:1006B0000044025800ED00E02DE9F04F93B0B44B38
:1006C0002022FF2100900AA89D6800F0EFFBB14AAC
:1006D0001378A3B90121B04811700360302383F36C
:1006E000118803680BB101F067FA0023AB4A4FF49D
:1006F0007A71A94801F056FA002383F31188009B10
:1007000013B1A74B009A1A60A64A1378032B03D0A3
:1007100000231370A24A53604FF0000A009CD34696
:100720005646D146012000F089FB24B19C4B1B6842
:10073000002B00F02682002000F094FA0390039B27
:10074000002BF2DB012000F06FFB039B213B1F2BF2
:10075000E8D801A252F823F0D907000801080008E0
:100760009508000825070008250700082507000848
:1007700027090008F70A0008110A0008730A000890
:100780009B0A0008C10A000825070008D30A0008D0
:1007900025070008450B0008790800082507000810
:1007A000890B0008E50700087908000825070008FC
:1007B000730A000825070008250700082507000818
:1007C0002507000825070008250700082507000859
:1007D00025070008950800080220FFF759FE0028A9
:1007E00040F0F981009B022105A8BAF1000F08BF73
:1007F0001C4641F21233ADF8143000F051FA91E783
:100800004FF47A7000F02EFA071EEBDB0220FFF7A0
:100810003FFE0028E6D0013F052F00F2DE81DFE831
:1008200007F0030A0D1013360523042105A80593CC
:1008300000F036FA17E004215548F9E704215A4838
:10084000F6E704215948F3E74FF01C08404608F149
:10085000040800F05DFA0421059005A800F020FAD4
:10086000B8F12C0FF2D101204FF0000900FA07F780
:1008700047EA0B0B5FFA8BFB00F064FB26B10BF031
:100880000B030B2B08BF0024FFF70AFE4AE70421E5
:100890004748CDE7002EA5D00BF00B030B2BA1D1C1
:1008A0000220FFF7F5FD074600289BD00120002617
:1008B00000F02CFA0220FFF73BFE1FFA86F84046B4
:1008C00000F034FA0446B0B1039940460136A1F174
:1008D00040025142514100F039FA0028EDD1BA46A8
:1008E000044641F21213022105A83E46ADF8143029
:1008F00000F0D6F916E725460120FFF719FE244B34
:100900009B68AB4207D9284600F002FA013040F05C
:1009100067810435F3E70025224BBA463E461D7039
:100920001F4B5D60A8E7002E3FF45CAF0BF00B039C
:100930000B2B7FF457AF0220FFF7FAFD322000F0B7
:1009400091F9B0F10008FFF64DAF18F003077FF4FE
:1009500049AF0F4A08EB0503926893423FF642AF56
:10096000B8F5807F3FF73EAF124BB845019323DDCA
:100970004FF47A7000F076F90390039A002AFFF69C
:1009800031AF039A0137019B03F8012BEDE700BF5C
:10099000002200207C23002060220020B9040008EF
:1009A000802300207822002004220020082200203A
:1009B0000C2200207C220020C820FFF769FD07469A
:1009C00000283FF40FAF1F2D11D8C5F120020AAB4C
:1009D00025F0030084494245184428BF424601924D
:1009E00000F03EFA019AFF217F4800F05FFA4FEADB
:1009F000A803C8F387027C492846019300F05EFAF9
:100A0000064600283FF46DAF019B05EB830533E7F5
:100A10000220FFF73DFD00283FF4E4AE00F0B4F9FA
:100A200000283FF4DFAE0027B846704B9B68BB42FE
:100A300018D91F2F11D80A9B01330ED027F00303BA
:100A400012AA134453F8203C05934046042205A9FA
:100A5000043700F0ADFA8046E7E7384600F058F971
:100A60000590F2E7CDF81480042105A800F018F9EC
:100A700002E70023642104A8049300F007F900288A
:100A80007FF4B0AE0220FFF703FD00283FF4AAAECA
:100A9000049800F06FF90590E6E70023642104A8AC
:100AA000049300F0F3F800287FF49CAE0220FFF7D7
:100AB000EFFC00283FF496AE049800F05DF9EAE7F9
:100AC0000220FFF7E5FC00283FF48CAE00F06CF943
:100AD000E1E70220FFF7DCFC00283FF483AE05A924
:100AE000142000F067F907460421049004A800F0E0
:100AF000D7F83946B9E7322000F0B4F8071EFFF600
:100B000071AEBB077FF46EAE384A07EB09039268FB
:100B100093423FF667AE0220FFF7BAFC00283FF48D
:100B200061AE27F003074F44B9453FF4A5AE4846F0
:100B300009F1040900F0ECF80421059005A800F083
:100B4000AFF8F1E74FF47A70FFF7A2FC00283FF40A
:100B500049AE00F019F9002844D00A9B01330BD0AC
:100B600008220AA9002000F0A9F900283AD0202282
:100B7000FF210AA800F09AF9FFF792FC1C4800F048
:100B800055FF13B0BDE8F08F002E3FF42BAE0BF0F5
:100B90000B030B2B7FF426AE0023642105A80593DD
:100BA00000F074F8074600287FF41CAE0220FFF71F
:100BB0006FFC804600283FF415AEFFF771FC41F250
:100BC000883000F033FF059800F0F0F946463C46C7
:100BD00000F0B8F9A6E506464EE64FF0000901E63A
:100BE000BA467EE637467CE67C22002000220020C2
:100BF000A0860100704700000F4B70B51B780C46B3
:100C00000133DBB2012B11D80C4D4FF47A732968F4
:100C1000A2FB033222460E6A01462846B0478442B0
:100C200004D1074B002201201A7070BD4FF4FA70F6
:100C300000F0FCFE0020F8E710220020282600200B
:100C4000B423002070B504464FF47A76412C254633
:100C500028BF412506FB05F000F0E8FE641BF5D136
:100C600070BD0000002307B5024601210DF1070009
:100C70008DF80730FFF7C0FF20B19DF8070003B0E3
:100C80005DF804FB4FF0FF30F9E700000A4604214D
:100C900008B5FFF7B1FF80F00100C0B2404208BDC7
:100CA00030B4054C0A46014623682046DD69034BF3
:100CB000AC4630BC604700BF28260020A08601005B
:100CC00070B5104C0025104E01F0CCF92080306832
:100CD000238883420CD800252088013801F0BEF912
:100CE00023880544013BB5F5802F2380F4D370BDE4
:100CF00001F0B4F9336805440133B5F5003F3360C2
:100D0000E5D3E8E7B62300208823002001F078BA75
:100D100000F1006000F500300068704700F10060ED
:100D2000920000F5003001F0F9B90000054B1A6897
:100D3000054B1B889B1A834202D9104401F08EB9DF
:100D40000020704788230020B623002038B50446D1
:100D5000074D29B128682044BDE8384001F096B914
:100D60002868204401F080F90028F3D038BD00BF86
:100D7000882300200020704700F1FF5000F58F10FD
:100D8000D0F8000870470000064991F8243033B1CC
:100D900000230822086A81F82430FFF7BFBF012032
:100DA000704700BF8C230020014B1868704700BFBC
:100DB0000010005C194B01380322084470B51D680F
:100DC000174BC5F30B042D0C1E88A6420BD15C6893
:100DD0000A46013C824213460FD214F9016F4EB10C
:100DE00002F8016BF6E7013A03F10803ECD1814206
:100DF0000B4602D22C2203F8012B0424094A168840
:100E0000AE4204D1984284BF967803F8016B013C4E
:100E100002F10402F3D1581A70BD00BF0010005C4B
:100E200014220020503B0008022803D1024B4FF44B
:100E300000229A61704700BF00100258022802D1B8
:100E4000014B08229A61704700100258022804D111
:100E5000024A536983F00803536170470010025837
:100E6000002310B5934203D0CC5CC4540133F9E79E
:100E700010BD0000013810B510F9013F3BB191F9E8
:100E800000409C4203D11AB10131013AF4E71AB192
:100E900091F90020981A10BD1046FCE7034602465F
:100EA000D01A12F9011B0029FAD1704702440346F7
:100EB000934202D003F8011BFAE770472DE9F8438B
:100EC0001F4D14460746884695F8242052BBDFF88C
:100ED00070909CB395F824302BB92022FF2148460E
:100EE0002F62FFF7E3FF95F824004146C0F10802A6
:100EF00005EB8000A24228BF2246D6B29200FFF73F
:100F0000AFFF95F82430A41B17441E449044E4B26C
:100F1000F6B2082E85F82460DBD1FFF735FF0028F4
:100F2000D7D108E02B6A03EB82038342CFD0FFF7CF
:100F30002BFF0028CBD10020BDE8F8830120FBE780
:100F40008C230020024B1A78024B1A70704700BFA6
:100F5000B42300201022002010B5114C114800F0DD
:100F6000B9F821460F4800F0E1F824684FF47A7090
:100F7000D4F89020D2F8043843F00203C2F80438C1
:100F8000FFF760FE0849204600F0DEF9D4F8902013
:100F9000D2F8043823F00203C2F8043810BD00BFB1
:100FA0000C3C000828260020143C00087047000074
:100FB00030B50A44084D91420DD011F8013B58401C
:100FC000082340F30004013B2C4013F0FF0384EAA4
:100FD0005000F6D1EFE730BD2083B8ED02684368DA
:100FE0001143016003B118477047000013B5406B0F
:100FF00000F58054D4F8A4381A681178042914D163
:10100000017C022911D11979012312898B401342E5
:101010000BD101A94C3002F059F8D4F8A44802468B
:10102000019B2179206800F0DFF902B010BD0000BB
:10103000143001F0DBBF00004FF0FF33143001F03B
:10104000D5BF00004C3002F0ADB800004FF0FF33C8
:101050004C3002F0A7B80000143001F0A9BF000026
:101060004FF0FF31143001F0A3BF00004C3002F00C
:1010700079B800004FF0FF324C3002F073B8000036
:101080000020704710B500F58054D4F8A4381A68D1
:101090001178042917D1017C022914D1597901232F
:1010A00052898B4013420ED1143001F03BFF0246AF
:1010B00048B1D4F8A4484FF4407361792068BDE882
:1010C000104000F07FB910BD406BFFF7DBBF0000A0
:1010D000704700007FB5124B0125042604460360CB
:1010E0000023057400F1840243602946C0E90233FD
:1010F0000C4B0290143001934FF44073009601F0B2
:10110000EDFE094B04F69442294604F14C0002948A
:10111000CDE900634FF4407301F0B4FF04B070BD3B
:10112000603B0008C9100008ED0F00080A68302372
:1011300083F311880B790B3342F823004B79133377
:1011400042F823008B7913B10B3342F8230000F5EA
:101150008053C3F8A41802230374002080F311887D
:101160007047000038B5037F044613B190F854303F
:10117000ABB90125201D0221FFF730FF04F1140057
:101180006FF00101257700F079FC04F14C0084F840
:1011900054506FF00101BDE8384000F06FBC38BD1D
:1011A00010B5012104460430FFF718FF0023237710
:1011B00084F8543010BD000038B5044600251430C2
:1011C00001F0A4FE04F14C00257701F073FF201D0F
:1011D00084F854500121FFF701FF2046BDE8384054
:1011E000FFF750BF90F8803003F06003202B06D14A
:1011F00090F881200023212A03D81F2A06D8002036
:101200007047222AFBD1C0E91D3303E0034A42673D
:1012100007228267C3670120704700BF2C2200208D
:1012200037B500F58055D5F8A4381A681178042927
:101230001AD1017C022917D11979012312898B4017
:10124000134211D100F14C04204601F0F3FF58B1D4
:1012500001A9204601F03AFFD5F8A4480246019BB7
:101260002179206800F0C0F803B030BD01F10B0314
:10127000F0B550F8236085B004460D46FEB130232A
:1012800083F3118804EB8507301D0821FFF7A6FEC4
:10129000FB6806F14C005B691B681BB1019001F013
:1012A00023FF019803A901F011FF024648B1039BF7
:1012B0002946204600F098F8002383F3118805B0F2
:1012C000F0BDFB685A691268002AF5D01B8A013B01
:1012D0001340F1D104F18002EAE70000133138B580
:1012E00050F82140ECB1302383F3118804F580538A
:1012F000D3F8A4281368527903EB8203DB689B6957
:101300005D6845B104216018FFF768FE294604F1C5
:10131000140001F011FE2046FFF7B4FE002383F312
:10132000118838BD7047000001F0C8B80123402281
:10133000002110B5044600F8303BFFF7B7FD00234D
:10134000C4E9013310BD000010B53023044683F317
:1013500011882422416000210C30FFF7A7FD2046B0
:1013600001F0CEF802230020237080F3118810BD15
:1013700070B500EB8103054650690E461446DA60ED
:1013800018B110220021FFF791FDA06918B11022B9
:101390000021FFF78BFD31462846BDE8704001F083
:1013A000B5B9000083682022002103F0011310B5B5
:1013B000044683601030FFF779FD2046BDE81040F9
:1013C00001F030BAF0B4012500EB810447898D406B
:1013D000E4683D43A469458123600023A260636003
:1013E000F0BC01F04DBA0000F0B4012500EB81041F
:1013F00007898D40E4683D436469058123600023CB
:10140000A2606360F0BC01F0C3BA000070B50223B3
:1014100000250446242203702946C0F888500C3069
:1014200040F8045CFFF742FD204684F8705001F05C
:1014300001F963681B6823B129462046BDE8704066
:10144000184770BD0378052B10B504460AD080F804
:101450008C300523037043681B680BB10421984747
:101460000023A36010BD00000178052906D190F883
:101470008C20436802701B6803B118477047000056
:1014800070B590F87030044613B1002380F87030C6
:1014900004F18002204601F0E9F963689B68B3B962
:1014A00094F8803013F0600535D00021204601F01B
:1014B000DBFC0021204601F0CBFC63681B6813B104
:1014C000062120469847062384F8703070BD2046D8
:1014D00098470028E4D0B4F88630A26F9A4288BFBB
:1014E000A36794F98030A56F002B4FF0300380F292
:1014F0000381002D00F0F280092284F8702083F32C
:10150000118800212046D4E91D23FFF76DFF002339
:1015100083F31188DAE794F8812003F07F0343EA2C
:10152000022340F20232934200F0C58021D8B3F585
:10153000807F48D00DD8012B3FD0022B00F0938044
:10154000002BB2D104F1880262670222A267E3672E
:10155000C1E7B3F5817F00F09B80B3F5407FA4D154
:1015600094F88230012BA0D1B4F8883043F0020304
:1015700032E0B3F5006F4DD017D8B3F5A06F31D07E
:10158000A3F5C063012B90D86368204694F88220AD
:101590005E6894F88310B4F88430B047002884D093
:1015A000436863670368A3671AE0B3F5106F36D02A
:1015B00040F6024293427FF478AF5C4B63670223AC
:1015C000A3670023C3E794F88230012B7FF46DAF4B
:1015D000B4F8883023F00203A4F88830C4E91D551C
:1015E000E56778E7B4F88030B3F5A06F0ED194F8D2
:1015F0008230204684F88A3001F07AF863681B68EC
:1016000013B1012120469847032323700023C4E926
:101610001D339CE704F18B0363670123C3E7237841
:10162000042B10D1302383F311882046FFF7BAFE34
:1016300085F311880321636884F88B5021701B683F
:101640000BB12046984794F88230002BDED084F806
:101650008B300423237063681B68002BD6D00221D3
:1016600020469847D2E794F8843020461D0603F0C0
:101670000F010AD501F0ECF8012804D002287FF40C
:1016800014AF2B4B9AE72B4B98E701F0D3F8F3E715
:1016900094F88230002B7FF408AF94F8843013F074
:1016A0000F01B3D01A06204602D501F0F5FBADE7D5
:1016B00001F0E6FBAAE794F88230002B7FF4F5AE48
:1016C00094F8843013F00F01A0D01B06204602D5F9
:1016D00001F0CAFB9AE701F0BBFB97E7142284F8FC
:1016E000702083F311882B462A4629462046FFF7AF
:1016F00069FE85F31188E9E65DB1152284F8702052
:1017000083F3118800212046D4E91D23FFF75AFEF8
:10171000FDE60B2284F8702083F311882B462A46BD
:1017200029462046FFF760FEE3E700BF903B000834
:10173000883B00088C3B000838B590F870300446B0
:10174000002B3ED0063BDAB20F2A34D80F2B32D80A
:10175000DFE803F0373131082232313131313131B4
:1017600031313737856FB0F886309D4214D2C36867
:101770001B8AB5FBF3F203FB12556DB9302383F3DB
:1017800011882B462A462946FFF72EFE85F311883D
:101790000A2384F870300EE0142384F8703030236C
:1017A00083F31188002320461A461946FFF70AFEE4
:1017B000002383F3118838BDC36F03B1984700231A
:1017C000E7E70021204601F04FFB0021204601F011
:1017D0003FFB63681B6813B1062120469847062328
:1017E000D7E7000010B590F870300446142B29D0CC
:1017F00017D8062B05D001D81BB110BD093B022B11
:10180000FBD80021204601F02FFB0021204601F0EB
:101810001FFB63681B6813B1062120469847062307
:1018200019E0152BE9D10B2380F87030302383F3B6
:10183000118800231A461946FFF7D6FD002383F3CB
:101840001188DAE7C3689B695B68002BD5D1C36F49
:1018500003B19847002384F87030CEE700238268F4
:10186000037503691B6899689142FBD25A6803604B
:1018700042601060586070470023826803750369F6
:101880001B6899689142FBD85A68036042601060F7
:101890005860704708B50846302383F311880B7DE4
:1018A000032B05D0042B0DD02BB983F3118808BD71
:1018B0008B6900221A604FF0FF338361FFF7CEFF80
:1018C0000023F2E7D1E9003213605A60F3E7000029
:1018D000FFF7C4BF054BD9680875186802685360E4
:1018E0001A600122D8600275FEF78CBDB823002073
:1018F0000C4B30B5DD684B1C87B004460FD02B462F
:10190000094A684600F04EF92046FFF7E3FF009BC6
:1019100013B1684600F050F9A86907B030BDFFF771
:10192000D9FFF9E7B823002095180008044B1A687E
:10193000DB6890689B68984294BF00200120704744
:10194000B8230020084B10B51C68D8682268536083
:101950001A600122DC602275FFF78EFF01462046E7
:10196000BDE81040FEF74EBDB823002038B5074C47
:1019700001230025064907482370656001F098FCA3
:101980000223237085F3118838BD00BF2026002074
:10199000983B0008B823002000F044B9034A51687E
:1019A00053685B1A9842FBD8704700BF001000E0F4
:1019B0008B600223086108468B8270478368A3F11D
:1019C000840243F8142C026943F8442C426943F81A
:1019D000402C094A43F8242CC268A3F1200043F8A4
:1019E000182C022203F80C2C002203F80B2C034ABB
:1019F00043F8102C704700BF1D040008B8230020D6
:101A000008B5FFF7DBFFBDE80840FFF761BF000046
:101A1000024BDB6898610F20FFF75CBFB823002002
:101A2000302383F31188FFF7F3BF000008B50146A8
:101A3000302383F311880820FFF75AFF002383F334
:101A4000118808BD064BDB6839B1426818605A60DE
:101A5000136043600420FFF74BBF4FF0FF30704727
:101A6000B82300200368984206D01A6802605060CC
:101A700018469961FFF72CBF7047000038B504463F
:101A80000D462068844200D138BD036823605C6045
:101A90008561FFF71DFFF4E7036810B59C68A2425B
:101AA0000CD85C688A600B604C6021605960996852
:101AB0008A1A9A604FF0FF33836010BD121B1B68B7
:101AC000ECE700000A2938BF0A2170B504460D462C
:101AD0000A26601901F0E4FB01F0CCFB041BA542CF
:101AE00003D8751C04462E46F3E70A2E04D90120BC
:101AF000BDE8704001F01CBC70BD0000F8B5144B8F
:101B00000D460A2A4FF00A07D96103F110018260DD
:101B100038BF0A22416019691446016048601861A3
:101B2000A81801F0ADFB01F0A5FB431B0646A3423C
:101B300006D37C1C28192746354601F0B1FBF2E795
:101B40000A2F04D90120BDE8F84001F0F1BBF8BD2F
:101B5000B8230020F8B506460D4601F08BFB0F4A6E
:101B6000134653F8107F9F4206D12A46014630465D
:101B7000BDE8F840FFF7C2BFD169BB68441A2C1911
:101B800028BF2C46A34202D92946FFF79BFF2246D5
:101B900031460348BDE8F840FFF77EBFB823002078
:101BA000C8230020C0E90323002310B45DF8044BD0
:101BB0004361FFF7CFBF000010B5194C236998426D
:101BC0000DD08168D0E9003213605A609A680A44E7
:101BD0009A60002303604FF0FF33A36110BD0268D9
:101BE000234643F8102F53600022026022699A4274
:101BF00003D1BDE8104001F04DBB936881680B44F0
:101C0000936001F037FB2269E1699268441AA242AD
:101C1000E4D91144BDE81040091AFFF753BF00BFD3
:101C2000B82300202DE9F047DFF8BC8008F1100749
:101C30002C4ED8F8105001F01DFBD8F81C40AA68B3
:101C4000031B9A423ED814444FF00009D5E90032F4
:101C5000C8F81C4013605A60C5F80090D8F81030DE
:101C6000B34201D101F016FB89F31188D5E90331A4
:101C700028469847302383F311886B69002BD8D00E
:101C800001F0F8FA6A69A0EB040982464A450DD2D0
:101C9000022001F04DFB0022D8F81030B34208D1E9
:101CA00051462846BDE8F047FFF728BF121A2244E4
:101CB000F2E712EB09092946384638BF4A46FFF7D2
:101CC000EBFEB5E7D8F81030B34208D01444C8F89A
:101CD0001C00211AA960BDE8F047FFF7F3BEBDE87C
:101CE000F08700BFC8230020B823002000207047E1
:101CF000FEE70000704700004FF0FF307047000023
:101D000002290CD0032904D00129074818BF00205C
:101D10007047032A05D8054800EBC2007047044805
:101D200070470020704700BF703C00083C22002034
:101D3000243C000870B59AB005460846144601A92F
:101D400000F0C2F801A8FFF7A9F8431C0022C6B2B0
:101D50005B001046C5E9003423700323023404F805
:101D6000013C01ABD1B202348E4201D81AB070BD31
:101D700013F8011B013204F8010C04F8021CF1E70E
:101D800008B5302383F311880348FFF749FA00238D
:101D900083F3118808BD00BF2826002090F880300A
:101DA00003F01F02012A07D190F881200B2A03D1EA
:101DB0000023C0E91D3315E003F06003202B08D198
:101DC000B0F884302BB990F88120212A03D81F2A3B
:101DD00004D8FFF707BA222AEBD0FAE7034A426792
:101DE00007228267C3670120704700BF33220020AB
:101DF00007B5052917D8DFE801F0191603191920CE
:101E0000302383F31188104A01210190FFF7B0FAC3
:101E1000019802210D4AFFF7ABFA0D48FFF7CCF904
:101E2000002383F3118803B05DF804FB302383F3B0
:101E300011880748FFF796F9F2E7302383F31188FA
:101E40000348FFF7ADF9EBE7C43B0008E83B0008A7
:101E50002826002038B50C4D0C4C2A460C4904F1BC
:101E60000800FFF767FF05F1CA0204F110000949F5
:101E7000FFF760FF05F5CA7204F118000649BDE8D6
:101E80003840FFF757BF00BF003F00203C22002032
:101E9000A43B0008AE3B0008B93B000870B50446FF
:101EA00008460D46FEF7FAFFC6B220460134037815
:101EB0000BB9184670BD32462946FEF7DBFF0028F5
:101EC000F3D10120F6E700002DE9F04705460C4666
:101ED000FEF7E4FF2B49C6B22846FFF7DFFF08B143
:101EE0000B36F6B228492846FFF7D8FF08B110365E
:101EF000F6B2632E0BD8DFF88C80DFF88C90234F7E
:101F0000DFF894A02E7846B92670BDE8F087294600
:101F10002046BDE8F04701F0FDBD252E2ED1072259
:101F200041462846FEF7A6FF70B9194B224603F139
:101F3000100153F8040B8B4242F8040BF9D11B88B3
:101F4000073512341380DDE7082249462846FEF79C
:101F500091FF98B9A21C0F4B197802320909C95D8B
:101F600002F8041C13F8011B01F00F015345C95D71
:101F700002F8031CF0D118340835C3E7013504F822
:101F8000016BBFE7903C0008B93B0008AB3C000880
:101F9000983C000800E8F11F0CE8F11FBFF34F8FD9
:101FA000044B1A695107FCD1D3F810215207F8D11C
:101FB000704700BF0020005208B50D4B1B78ABB92D
:101FC000FFF7ECFF0B4BDA68D10704D50A4A5A60D9
:101FD00002F188325A60D3F80C21D20706D5064A9E
:101FE000C3F8042102F18832C3F8042108BD00BF00
:101FF0005E410020002000522301674508B5114BC7
:102000001B78F3B9104B1A69510703D5DA6842F00F
:102010004002DA60D3F81021520705D5D3F80C211D
:1020200042F04002C3F80C21FFF7B8FF064BDA6814
:1020300042F00102DA60D3F80C2142F00102C3F849
:102040000C2108BD5E410020002000520F289ABFDD
:1020500000F5806040040020704700004FF400301D
:1020600070470000102070470F2808B50BD8FFF705
:10207000EDFF00F500330268013204D104308342E1
:10208000F9D1012008BD0020FCE700000F2838B579
:1020900005463FD8FFF782FF1F4CFFF78DFF4FF03B
:1020A000FF3307286361C4F814311DD82361FFF79B
:1020B00075FF030243F02403E360E36843F0800309
:1020C000E36023695A07FCD42846FFF767FFFFF750
:1020D000BDFF4FF4003100F0F5F82846FFF78EFF02
:1020E000BDE83840FFF7C0BFC4F81031FFF756FF16
:1020F000A0F108031B0243F02403C4F80C31D4F808
:102100000C3143F08003C4F80C31D4F810315B0774
:10211000FBD4D9E7002038BD002000522DE9F84F4C
:1021200005460C46104645EA0203DE0602D00020B2
:10213000BDE8F88F20F01F00DFF8BCB0DFF8BCA0CE
:10214000FFF73AFF04EB0008444503D10120FFF7F5
:1021500055FFEDE720222946204601F0CBFC10B9BF
:1021600020352034F0E72B4605F120021F68791C4A
:10217000DDD104339A42F9D105F178431B481C4E56
:10218000B3F5801F1B4B38BF184603F1F80332BF6D
:10219000D946D1461E46FFF701FF0760A5EB040CA8
:1021A000336804F11C0143F002033360231FD9F8A4
:1021B000007017F00507FAD153F8042F8B424CF842
:1021C0000320F4D1BFF34F8FFFF7E8FE4FF0FF334A
:1021D0002022214603602846336823F0020333603F
:1021E00001F088FC0028BBD03846B0E7142100522B
:1021F0000C200052142000521020005210210052D6
:1022000010B5084C237828B11BB9FFF7D5FE012380
:10221000237010BD002BFCD02070BDE81040FFF7EC
:10222000EDBE00BF5E4100200244074BD2B210B5A4
:10223000904200D110BD441C00B253F8200041F878
:10224000040BE0B2F4E700BF504000580E4B30B52D
:102250001C6F240405D41C6F1C671C6F44F40044DD
:102260001C670A4C02442368D2B243F48073236093
:10227000074B904200D130BD441C51F8045B00B2C2
:1022800043F82050E0B2F4E70044025800480258F6
:102290005040005807B5012201A90020FFF7C4FFF4
:1022A000019803B05DF804FB13B50446FFF7F2FF95
:1022B000A04205D0012201A900200194FFF7C6FF2A
:1022C00002B010BD0144BFF34F8F064B884204D3C8
:1022D000BFF34F8FBFF36F8F7047C3F85C0220309E
:1022E000F4E700BF00ED00E0034B1A681AB9034A97
:1022F000D2F8D0241A607047604100200040025894
:1023000008B5FFF7F1FF024B1868C0F3806008BD05
:102310006041002070B5BFF34F8FBFF36F8F1A4A33
:102320000021C2F85012BFF34F8FBFF36F8F536974
:1023300043F400335361BFF34F8FBFF36F8FC2F885
:102340008410BFF34F8FD2F8803043F6E074C3F3AC
:10235000C900C3F34E335B0103EA0406014646EAB3
:1023600081750139C2F86052F9D2203B13F1200F78
:10237000F2D1BFF34F8F536943F480335361BFF3FE
:102380004F8FBFF36F8F70BD00ED00E0FEE70000E0
:10239000214B2248224A70B5904237D3214BC11EAF
:1023A000DA1C121A22F003028B4238BF00220021ED
:1023B000FEF77CFD1C4A0023C2F88430BFF34F8F28
:1023C000D2F8803043F6E074C3F3C900C3F34E3350
:1023D0005B0103EA0406014646EA81750139C2F849
:1023E0006C52F9D2203B13F1200FF2D1BFF34F8F83
:1023F000BFF36F8FBFF34F8FBFF36F8F0023C2F810
:102400005032BFF34F8FBFF36F8F70BD53F8041B73
:1024100040F8041BC0E700BF943E0008344300208E
:10242000344300203443002000ED00E0074BD3F894
:10243000D81021EA0001C3F8D810D3F8002122EA0D
:102440000002C3F80021D3F800317047004402585D
:1024500070B5D0E9244300224FF0FF359E6804EBAD
:1024600042135101D3F80009002805DAD3F8000916
:1024700040F08040C3F80009D3F8000B002805DACB
:10248000D3F8000B40F08040C3F8000B0132631812
:102490009642C3F80859C3F8085BE0D24FF0011325
:1024A000C4F81C3870BD0000890141F020010161B1
:1024B00003699B06FCD41220FFF770BA10B50A4CD2
:1024C0002046FEF733FF094BC4F89030084BC4F8A0
:1024D0009430084C2046FEF729FF074BC4F8903093
:1024E000064BC4F8943010BD644100200000084041
:1024F000E03C00080042002000000440EC3C0008E2
:1025000070B503780546012B5CD1434BD0F8904061
:10251000984258D1414B0E216520D3F8D82042F083
:102520000062C3F8D820D3F8002142F00062C3F85B
:102530000021D3F80021D3F8802042F00062C3F8D4
:102540008020D3F8802022F00062C3F88020D3F8E6
:10255000803000F0ADFC324BE360324BC4F8003801
:102560000023D5F89060C4F8003EC02323604FF4E8
:102570000413A3633369002BFCDA01230C203361BD
:10258000FFF70CFA3369DB07FCD41220FFF706FAD9
:102590003369002BFCDA00262846A660FFF758FFB7
:1025A0006B68C4F81068DB68C4F81468C4F81C6869
:1025B00083BB1D4BA3614FF0FF336361A36843F0FE
:1025C0000103A36070BD194B9842C9D1134B4FF062
:1025D0008060D3F8D82042F00072C3F8D820D3F836
:1025E000002142F00072C3F80021D3F80021D3F893
:1025F000802042F00072C3F88020D3F8802022F0BF
:102600000072C3F88020D3F88030FFF70FFF0E214F
:102610004D209EE7064BCDE7644100200044025860
:102620004014004003002002003C30C00042002063
:10263000083C30C0F8B5D0F89040054600214FF076
:1026400000662046FFF730FFD5F8941000234FF0C6
:1026500001128F684FF0FF30C4F83438C4F81C28DA
:1026600004EB431201339F42C2F80069C2F8006BC9
:10267000C2F80809C2F8080BF2D20B68D5F890200E
:10268000C5F89830636210231361166916F01006BE
:10269000FBD11220FFF782F9D4F8003823F4FE634F
:1026A000C4F80038A36943F4402343F01003A36146
:1026B0000923C4F81038C4F814380B4BEB604FF002
:1026C000C043C4F8103B094BC4F8003BC4F8106980
:1026D000C4F80039D5F8983003F1100243F48013A0
:1026E000C5F89820A362F8BDBC3C000840800010EB
:1026F000D0F8902090F88A10D2F8003823F4FE63C6
:1027000043EA0113C2F80038704700002DE9F8438E
:1027100000EB8103D0F890500C468046DA680FFA3F
:1027200081F94801166806F00306731E022B05EBBB
:1027300041134FF0000194BFB604384EC3F8101B8C
:102740004FF0010104F1100398BF06F1805601FA21
:1027500003F3916998BF06F5004600293AD0578ADD
:1027600004F15801374349016F50D5F81C180B4349
:102770000021C5F81C382B180127C3F81019A740F1
:102780005369611E9BB3138A928B9B08012A88BFF1
:102790005343D8F89820981842EA034301F14002C5
:1027A0002146C8F89800284605EB82025360FFF7DF
:1027B0007BFE08EB8900C3681B8A43EA84534834D4
:1027C0001E4364012E51D5F81C381F43C5F81C78F0
:1027D000BDE8F88305EB4917D7F8001B21F4004149
:1027E000C7F8001BD5F81C1821EA0303C0E704F161
:1027F0003F030B4A2846214605EB83035A60FFF747
:1028000053FE05EB4910D0F8003923F40043C0F81B
:102810000039D5F81C3823EA0707D7E700800010F5
:1028200000040002D0F894201268C0F89820FFF746
:102830000FBE00005831D0F8903049015B5813F4B6
:10284000004004D013F4001F0CBF02200120704789
:102850004831D0F8903049015B5813F4004004D05F
:1028600013F4001F0CBF02200120704700EB810110
:10287000CB68196A0B6813604B685360704700009F
:1028800000EB810330B5DD68AA691368D36019B91C
:10289000402B84BF402313606B8A1468D0F89020CB
:1028A0001C4402EB4110013C09B2B4FBF3F4634356
:1028B000033323F0030343EAC44343F0C043C0F8A7
:1028C000103B2B6803F00303012B0ED1D2F808381C
:1028D00002EB411013F4807FD0F8003B14BF43F0AB
:1028E000805343F00053C0F8003B02EB4112D2F892
:1028F000003B43F00443C2F8003B30BD2DE9F041FA
:10290000D0F8906005460C4606EB4113D3F8087BDF
:102910003A07C3F8087B08D5D6F814381B0704D546
:1029200000EB8103DB685B689847FA071FD5D6F890
:102930001438DB071BD505EB8403D968CCB98B6948
:10294000488A5A68B2FBF0F600FB16228AB918686A
:10295000DA6890420DD2121AC3E90024302383F3BF
:10296000118821462846FFF78BFF84F31188BDE8C4
:10297000F081012303FA04F26B8923EA02036B81DD
:10298000CB68002BF3D021462846BDE8F04118471C
:1029900000EB81034A0170B5DD68D0F890306C69B6
:1029A0002668E66056BB1A444FF40020C2F81009AE
:1029B0002A6802F00302012A0AB20ED1D3F80808ED
:1029C00003EB421410F4807FD4F8000914BF40F0E8
:1029D000805040F00050C4F8000903EB4212D2F8D6
:1029E000000940F00440C2F800090122D3F834087D
:1029F00002FA01F10143C3F8341870BD19B9402E31
:102A000084BF4020206020681A442E8A8419013C2B
:102A1000B4FBF6F440EAC44040F00050C6E70000C2
:102A20002DE9F843D0F8906005460C464F0106EBBF
:102A30004113D3F8088918F0010FC3F808891CD096
:102A4000D6F81038DB0718D500EB8103D3F80CC09B
:102A5000DCF81430D3F800E0DA68964530D2A2EB07
:102A60000E024FF000091A60C3F80490302383F37C
:102A70001188FFF78DFF89F3118818F0800F1DD0A2
:102A8000D6F834380126A640334217D005EB84032C
:102A90000134D5F89050D3F80CC0E4B22F44DCF8E0
:102AA000142005EB0434D2F800E05168714514D3CA
:102AB000D5F8343823EA0606C5F83468BDE8F8834B
:102AC000012303FA01F2038923EA02030381DCF8FC
:102AD0000830002BD1D09847CFE7AEEB0103BCF80C
:102AE0001000834228BF0346D7F8180980B2B3EB21
:102AF000800FE3D89068A0F1040959F8048FC4F856
:102B00000080A0EB09089844B8F1040FF5D81844E8
:102B10000B4490605360C8E72DE9F84FD0F890500F
:102B200004466E69AB691E4016F480586E6103D08E
:102B3000BDE8F84FFEF76ABC002E12DAD5F8003E69
:102B40009B0705D0D5F8003E23F00303C5F8003EEF
:102B5000D5F80438204623F00103C5F80438FEF701
:102B600083FC370505D52046FFF772FC2046FEF7AB
:102B700069FCB0040CD5D5F8083813F0060FEB68E3
:102B800023F470530CBF43F4105343F4A053EB6091
:102B900031071BD56368DB681BB9AB6923F00803F9
:102BA000AB612378052B0CD1D5F8003E9A0705D0F0
:102BB000D5F8003E23F00303C5F8003E2046FEF79B
:102BC00053FC6368DB680BB120469847F30200F1C1
:102BD000BA80B70226D5D4F8909000274FF0010AAA
:102BE00009EB4712D2F8003B03F44023B3F5802FE2
:102BF00011D1D2F8003B002B0DDA62890AFA07F3F3
:102C000022EA0303638104EB8703DB68DB6813B10B
:102C10003946204698470137D4F89430FFB29B6874
:102C20009F42DDD9F00619D5D4F89000026AC2F3AC
:102C30000A1702F00F0302F4F012B2F5802F00F031
:102C4000CA80B2F5402F09D104EB8303002200F5BE
:102C50008050DB681B6A974240F0B0803003D5F8A3
:102C6000185835D5E90303D500212046FFF746FE65
:102C7000AA0303D501212046FFF740FE6B0303D5CD
:102C800002212046FFF73AFE2F0303D503212046F9
:102C9000FFF734FEE80203D504212046FFF72EFE9D
:102CA000A90203D505212046FFF728FE6A0203D5B5
:102CB00006212046FFF722FE2B0203D507212046DE
:102CC000FFF71CFEEF0103D508212046FFF716FE93
:102CD000700340F1A780E90703D500212046FFF7E4
:102CE0009FFEAA0703D501212046FFF799FE6B0737
:102CF00003D502212046FFF793FE2F0703D50321BA
:102D00002046FFF78DFEEE0603D504212046FFF78F
:102D100087FEA80603D505212046FFF781FE690638
:102D200003D506212046FFF77BFE2A0603D507219F
:102D30002046FFF775FEEB0574D520460821BDE857
:102D4000F84FFFF76DBED4F890904FF0000B4FF0A6
:102D5000010AD4F894305FFA8BF79B689F423FF6E4
:102D600038AF09EB4713D3F8002902F44022B2F53B
:102D7000802F20D1D3F80029002A1CDAD3F80029AB
:102D800042F09042C3F80029D3F80029002AFBDB67
:102D90003946D4F89000FFF787FB22890AFA07F337
:102DA00022EA0303238104EB8703DB689B6813B1EA
:102DB0003946204698470BF1010BCAE7910701D12C
:102DC000D0F80080072A02F101029CBF03F8018BB2
:102DD0004FEA18283FE704EB830300F58050DA68D8
:102DE000D2F818C0DCF80820DCE9001CA1EB0C0CC0
:102DF00000218F4208D1DB689B699A683A449A6047
:102E00005A683A445A6029E711F0030F01D1D0F80B
:102E100000808C4501F1010184BF02F8018B4FEA6B
:102E20001828E6E7BDE8F88F08B50348FFF774FEF9
:102E3000BDE8084000F07ABB6441002008B50348B3
:102E4000FFF76AFEBDE8084000F070BB00420020BA
:102E5000D0F8903003EB4111D1F8003B43F400135C
:102E6000C1F8003B70470000D0F8903003EB4111EF
:102E7000D1F8003943F40013C1F80039704700005D
:102E8000D0F8903003EB4111D1F8003B23F400134C
:102E9000C1F8003B70470000D0F8903003EB4111BF
:102EA000D1F8003923F40013C1F80039704700004D
:102EB000090100F16043012203F56143C9B283F8BF
:102EC000001300F01F039A4043099B0003F1604385
:102ED00003F56143C3F880211A60704730B50433AD
:102EE000039C0172002104FB0325C160C0E9065365
:102EF000049B0363059BC0E90000C0E90422C0E90C
:102F00000842C0E90A11436330BD00000022416A53
:102F1000C260C0E90411C0E90A226FF00101FEF7A6
:102F2000ADBD0000D0E90432934201D1C2680AB9B4
:102F3000181D704700207047036919600021C2689E
:102F40000132C260C269134482699342036124BFA3
:102F5000436A0361FEF786BD38B504460D46E36853
:102F60003BB162690020131D1268A3621344E3623F
:102F700007E0237A33B929462046FEF763FD00288F
:102F8000EDDA38BD6FF00100FBE70000C368C269ED
:102F9000013BC3604369134482699342436124BF88
:102FA000436A436100238362036B03B11847704790
:102FB00070B53023044683F31188866A3EB9FFF763
:102FC000CBFF054618B186F31188284670BDA36A69
:102FD000E26A13F8015B9342A36202D32046FFF733
:102FE000D5FF002383F31188EFE700002DE9F84FA8
:102FF00004460E46174698464FF0300989F311886B
:103000000025AA46D4F828B0BBF1000F09D14146EB
:103010002046FFF7A1FF20B18BF311882846BDE8B9
:10302000F88FD4E90A12A7EB050B521A934528BF73
:103030009346BBF1400F1BD9334601F1400251F8D2
:10304000040B914243F8040BF9D1A36A4036403592
:103050004033A362D4E90A239A4202D32046FFF701
:1030600095FF8AF31188BD42D8D289F31188C9E748
:1030700030465A46FDF7F4FEA36A5E445D445B4465
:10308000A362E7E710B5029C0433017203FB04213D
:10309000C460C0E906130023C0E90A33039B03633D
:1030A000049BC0E90000C0E90422C0E90842436370
:1030B00010BD0000026A6FF00101C260426AC0E9FF
:1030C00004220022C0E90A22FEF7D8BCD0E904237A
:1030D0009A4201D1C26822B9184650F8043B0B60ED
:1030E000704700231846FAE7C3680021C26901331C
:1030F000C3604369134482699342436124BF436AB6
:103100004361FEF7AFBC000038B504460D46E368E6
:103110003BB1236900201A1DA262E2691344E362F5
:1031200007E0237A33B929462046FEF78BFC0028B6
:10313000EDDA38BD6FF00100FBE7000003691960AC
:10314000C268013AC260C269134482699342036152
:1031500024BF436A036100238362036B03B11847F2
:103160007047000070B530230D460446114683F3C6
:103170001188866A2EB9FFF7C7FF10B186F3118850
:1031800070BDA36A1D70A36AE26A01339342A36211
:1031900004D3E16920460439FFF7D0FF002080F313
:1031A0001188EDE72DE9F84F04460D469046994603
:1031B0004FF0300A8AF311880026B346A76A4FB948
:1031C00049462046FFF7A0FF20B187F3118830461B
:1031D000BDE8F88FD4E90A073A1AA8EB0607974228
:1031E00028BF1746402F1BD905F1400355F8042B83
:1031F0009D4240F8042BF9D1A36A40364033A362C4
:10320000D4E90A239A4204D3E16920460439FFF73E
:1032100095FF8BF311884645D9D28AF31188CDE703
:1032200029463A46FDF71CFEA36A3D443E443B4412
:10323000A362E5E7D0E904239A4217D1C3689BB1A2
:10324000836A8BB1043B9B1A0ED01360C368013BA9
:10325000C360C3691A4483699A42026124BF436A06
:103260000361002383620123184670470023FBE7B4
:1032700000F086B9014B586A704700BF000C00404F
:10328000034B002258631A610222DA60704700BFC4
:10329000000C0040014B0022DA607047000C004037
:1032A000014B5863704700BF000C0040FEE7000070
:1032B00070B51B4B0025044686B058600E468562EB
:1032C000016300F00BF904F11003A560E562C4E9A5
:1032D00004334FF0FF33C4E90044C4E90635FFF777
:1032E000C9FF2B46024604F134012046C4E90823F5
:1032F00080230C4A2565FEF75BFB01230A4AE06048
:1033000000920375684672680192B268CDE90223A3
:10331000064BCDE90435FEF773FB06B070BD00BF68
:1033200020260020F83C0008FD3C0008AD320008D3
:10333000024AD36A1843D062704700BFB823002006
:103340004B6843608B688360CB68C3600B694361E3
:103350004B6903628B6943620B680360704700002E
:1033600008B53C4B40F2FF713B48D3F888200A4334
:10337000C3F88820D3F8882022F4FF6222F00702E5
:10338000C3F88820D3F88820D3F8E0200A43C3F894
:10339000E020D3F808210A43C3F808212F4AD3F8C4
:1033A00008311146FFF7CCFF00F5806002F11C01E7
:1033B000FFF7C6FF00F5806002F13801FFF7C0FF9C
:1033C00000F5806002F15401FFF7BAFF00F580605C
:1033D00002F17001FFF7B4FF00F5806002F18C018B
:1033E000FFF7AEFF00F5806002F1A801FFF7A8FF2C
:1033F00000F5806002F1C401FFF7A2FF00F58060D4
:1034000002F1E001FFF79CFF00F5806002F1FC0192
:10341000FFF796FF02F58C7100F58060FFF790FFD3
:1034200000F076F90E4BD3F8902242F00102C3F877
:103430009022D3F8942242F00102C3F8942205228C
:10344000C3F898204FF06052C3F89C20054AC3F897
:10345000A02008BD0044025800000258043D0008A6
:1034600000ED00E01F00080308B500F025FBFEF7A3
:103470007DFA0F4BD3F8DC2042F04002C3F8DC2089
:10348000D3F8042122F04002C3F80421D3F8043118
:10349000084B1A6842F008021A601A6842F00402E7
:1034A0001A60FEF721FFBDE80840FEF7D3BC00BF5D
:1034B000004402580018024870470000EFF30983E7
:1034C000054968334A6B22F001024A6383F3098895
:1034D000002383F31188704700EF00E0302080F371
:1034E000118862B60D4B0E4AD96821F4E0610904D7
:1034F000090C0A430B49DA60D3F8FC2042F08072D1
:10350000C3F8FC20084AC2F8B01F116841F001015D
:1035100011602022DA7783F82200704700ED00E086
:103520000003FA0555CEACC5001000E0302310B5FD
:1035300083F311880E4B5B6813F4006314D0F1EE33
:10354000103AEFF309844FF08073683CE361094B54
:10355000DB6B236684F30988FEF7E8F910B1064BAC
:10356000A36110BD054BFBE783F31188F9E700BFAA
:1035700000ED00E000EF00E02F0400083204000836
:10358000114BD3F8E82042F00802C3F8E820D3F842
:10359000102142F00802C3F810210C4AD3F8103170
:1035A000D36B43F00803D363C722094B9A624FF0F1
:1035B000FF32DA6200229A615A63DA605A600122AD
:1035C0005A611A60704700BF004402580010005C46
:1035D000000C0040094A08B51169D3680B40D9B204
:1035E0009B076FEA0101116107D5302383F311882E
:1035F000FEF7D2F9002383F3118808BD000C0040C8
:10360000064BD3F8DC200243C3F8DC20D3F80421B6
:103610001043C3F80401D3F8043170470044025842
:103620003A4B4FF0FF31D3F8802062F00042C3F8EC
:103630008020D3F8802002F00042C3F88020D3F825
:103640008020D3F88420C3F88410D3F8842000228B
:10365000C3F88420D3F88400D86F40F0FF4040F4D2
:10366000FF0040F4DF4040F07F00D867D86F20F0C3
:10367000FF4020F4FF0020F4DF4020F07F00D867F7
:10368000D86FD3F888006FEA40506FEA5050C3F803
:103690008800D3F88800C0F30A00C3F88800D3F884
:1036A0008800D3F89000C3F89010D3F89000C3F8C6
:1036B0009020D3F89000D3F89400C3F89410D3F876
:1036C0009400C3F89420D3F89400D3F89800C3F87A
:1036D0009810D3F89800C3F89820D3F89800D3F83E
:1036E0008C00C3F88C10D3F88C00C3F88C20D3F86E
:1036F0008C00D3F89C00C3F89C10D3F89C10C3F83E
:103700009C20D3F89C3000F0AFB900BF00440258B1
:1037100008B50122534BC3F80821534BD3F8F420CA
:1037200042F00202C3F8F420D3F81C2142F0020256
:10373000C3F81C210222D3F81C314C4BDA605A68C2
:103740009104FCD54A4A1A6001229A60494ADA601B
:1037500000221A614FF440429A61444B9A699204E4
:10376000FCD51A6842F480721A603F4B1A6F12F44B
:10377000407F04D04FF480321A6700221A671A681B
:1037800042F001021A60384B1A685007FCD500223B
:103790001A611A6912F03802FBD1012119604FF049
:1037A000804159605A67344ADA62344A1A611A68A9
:1037B00042F480321A602C4B1A689103FCD51A68C7
:1037C00042F480521A601A689204FCD52C4A2D49A2
:1037D0009A6200225A63196301F57C01DA6301F2EF
:1037E000E71199635A64284A1A64284ADA621A6807
:1037F00042F0A8521A601C4B1A6802F02852B2F12B
:10380000285FF9D148229A614FF48862DA61402238
:103810001A621F4ADA641F4A1A651F4A5A651F4A0C
:103820009A6532231E4A1360136803F00F03022BBC
:10383000FAD10D4A136943F003031361136903F0CE
:103840003803182BFAD14FF00050FFF7D9FE4FF094
:103850008040FFF7D5FE4FF00040BDE80840FFF77D
:10386000CFBE00BF008000510044025800480258FB
:1038700000C000F0020000010000FF010088900875
:103880001210200063020901470E0508DD0BBF017D
:1038900020000020000001100910E00000010110CC
:1038A000002000524FF0B04208B5D2F8883003F043
:1038B0000103C2F8883023B1044A13680BB1506881
:1038C0009847BDE80840FFF731BE00BFB442002072
:1038D0004FF0B04208B5D2F8883003F00203C2F8C6
:1038E000883023B1044A93680BB1D0689847BDE88B
:1038F0000840FFF71BBE00BFB44200204FF0B042AB
:1039000008B5D2F8883003F00403C2F8883023B138
:10391000044A13690BB150699847BDE80840FFF7A6
:1039200005BE00BFB44200204FF0B04208B5D2F847
:10393000883003F00803C2F8883023B1044A936941
:103940000BB1D0699847BDE80840FFF7EFBD00BF55
:10395000B44200204FF0B04208B5D2F8883003F0EE
:103960001003C2F8883023B1044A136A0BB1506ABD
:103970009847BDE80840FFF7D9BD00BFB44200201A
:103980004FF0B04310B5D3F8884004F47872C3F810
:103990008820A30604D5124A936A0BB1D06A9847CF
:1039A000600604D50E4A136B0BB1506B9847210685
:1039B00004D50B4A936B0BB1D06B9847E20504D545
:1039C000074A136C0BB1506C9847A30504D5044A01
:1039D000936C0BB1D06C9847BDE81040FFF7A6BDC3
:1039E000B44200204FF0B04310B5D3F8884004F43F
:1039F0007C42C3F88820620504D5164A136D0BB1CA
:103A0000506D9847230504D5124A936D0BB1D06DC4
:103A10009847E00404D50F4A136E0BB1506E9847D7
:103A2000A10404D50B4A936E0BB1D06E9847620483
:103A300004D5084A136F0BB1506F9847230404D57F
:103A4000044A936F0BB1D06F9847BDE81040FFF761
:103A50006DBD00BFB442002008B5FFF7BBFDBDE857
:103A60000840FFF763BD0000062108B50846FFF7D0
:103A70001FFA06210720FFF71BFA06210820FFF78F
:103A800017FA06210920FFF713FA06210A20FFF78B
:103A90000FFA06211720FFF70BFA06212820FFF75F
:103AA00007FA09217A20FFF703FA07213220BDE83F
:103AB0000840FFF7FDB9000008B5FFF7B1FD00F0C1
:103AC0000BF8FDF731FCFDF703FBFFF7F5FCBDE854
:103AD0000840FFF7CDBB00000023054A194601331B
:103AE000102BC2E9001102F10802F8D1704700BFA3
:103AF000B442002010B501390244904201D10020A7
:103B000005E0037811F8014FA34201D0181B10BD46
:103B10000130F2E7034611F8012B03F8012B002ACC
:103B2000F9D1704753544D333248373F3F3F00532C
:103B3000544D3332483733782F3732780053544D51
:103B40003332483734332F3735332F373530000091
:103B500001105A000310590001205800032056009C
:103B6000000000004D100008391000087510000812
:103B7000611000086D100008591000084510000879
:103B80003110000881100008000000000100000052
:103B90000000000063300000943B00081024002067
:103BA000202600204172647550696C6F74002542B4
:103BB0004F415244252D424C002553455249414C1A
:103BC0002500000002000000000000006D12000847
:103BD000DD12000840004000D03E0020E03E002002
:103BE00002000000000000000300000000000000D0
:103BF000251300080000000010000000F03E002027
:103C000000000000010000000000000064410020EE
:103C100001010200F11D0008011D00089D1D0008A2
:103C2000811D0008430000002C3C000809024300ED
:103C3000020100C032090400000102020100052453
:103C400000100105240100010424020205240600DD
:103C500001070582030800FF09040100020A0000B1
:103C60000007050102400000070581024000000036
:103C700012000000783C0008120110010200004010
:103C80000912415700020102030100000403090464
:103C900025424F4152442500416F636F64612D52AC
:103CA000432D483734334475616C0030313233343E
:103CB000353637383941424344454600000000005C
:103CC0008114000839170008E5170008400040007B
:103CD0009C4200209C42002001000000AC420020D9
:103CE000800000004001000008000000000100000A
:103CF00000100000080000006D61696E0069646CCE
:103D0000650000000000802A00000000AAAAAAAAFC
:103D100000000024FFFF00000000000000A00A00D7
:103D20000000000100000000AAAAAAAA00000001E9
:103D3000FFFF000000000000000000000000004045
:103D400000000000AAAAAAAA00000040FFFF00008D
:103D50000000000000000000400000000000000023
:103D6000AAAAAAAA40000000FFFF0000000000006D
:103D7000000000004000400000000000AAAAAAAA1B
:103D800000004000F7FF00000000000000000000FD
:103D90000000000000000000AAAAAAAA000000007B
:103DA000FFFF000000000000000000000000000015
:103DB00000000000AAAAAAAA00000000FFFF00005D
:103DC00000000000000000000000000000000000F3
:103DD000AAAAAAAA00000000FFFF0000000000003D
:103DE000000000000000000000000000AAAAAAAA2B
:103DF00000000000FFFF00000000000000000000C5
:103E00000000000000000000AAAAAAAA000000000A
:103E1000FFFF0000000000000000000000000000A4
:103E200000000000AAAAAAAA00000000FFFF0000EC
:103E300000000000000000005A1400000000000014
:103E400000001A0000000000FF0000000000000059
:103E5000243B0008830400002F3B000850040000AE
:103E60003D3B00080096000000000800960000009E
:103E700000080000040000008C3C00080000000066
:103E80000000000000000000000000000000000032
:043E9000000000002E
:00000001FF
